:1000000031C04BC065C349C048C047C046C045C0A9
:1000100044C043C042C041C040C03FC03EC00403D2
:1000200009041603550053004200740069006E0075
:10003000790053005000490012011001000000082F
:1000400081179F0C0401000200010902190001013F
:100050000080640904000001FF000000070581031F
:1000600008000A0011241FBECFE5D1E0DEBFCDBFDE
:1000700010E0A0E6B0E0ECEBF9E002C005900D92D4
:10008000A436B107D9F710E0A4E6B0E001C01D9294
:10009000AB3AB107E1F740D18FC4B2CFDC01FB012D
:1000A0006091600050E07D9190E040E820E030E019
:1000B000842F872309F0C09A062E00C0000000009C
:1000C00000000A94D1F7C29A062E00C0000000007A
:1000D00000000A94D1F7990FB1999F5FC098C29818
:1000E00046952F5F3F4F2830310511F790835F5FB2
:1000F000543011F03196D7CF089520916600309199
:1001000067002F5F3F4F30936700209366002150B8
:10011000304080916A0087FF02C0220F331F809316
:100120006B0020FF03C0886080936B00832F86954F
:1001300080936C003695279520936D008BE690E0B8
:100140006FE670E0ABDF08950F931F93CF93DF93BB
:10015000062FEC0110E005C0D0DF8091720089937A
:100160001F5F1017C8F3802FDF91CF911F910F9160
:1001700008958F929F92AF92BF92CF92DF92EF92AB
:10018000FF920F931F93CF93DF93862EA09068006A
:10019000B090690090906400C0906500209160006C
:1001A000E22EFF2425E0EE0CFF1C2A95E1F78C01DE
:1001B000DD2425C0F801808180936E009EDF809150
:1001C0006B0090E6892780936B00C0E0D0E011C0FF
:1001D0008BE690E06FE670E061DF909172008091B5
:1001E0006E00981721F4991511F09C1529F4CE0D85
:1001F000DF1DCA15DB0560F3D3940F5F1F4FD814C2
:10020000C8F281E0DF91CF911F910F91FF90EF90A5
:10021000DF90CF90BF90AF909F908F900895CF9335
:10022000DF93EC013981332331F490939000809374
:100230008F0088E06EC08C81E82FF0E0313041F40F
:1002400080818883D0939000C0938F0081E061C04B
:10025000323011F48A8112C0BE016E5F7F4F4A8135
:10026000242F277081E090E0982F01C0990F2A95E4
:10027000EAF7333029F4909580818923808343C045
:10028000343019F48081892BF9CF353049F440930B
:100290006000B99887B3856287BB88B3887D04C046
:1002A000363021F480E287BB88BB2DC0373049F45B
:1002B000CB01BE01F3DED0939000C0938F0084E0A9
:1002C00028C0383031F4409364008B8180936500FE
:1002D0001AC08C819D8190936700809366003930AD
:1002E00011F480E213C03B3011F480EA0FC08A8120
:1002F0009B8190936900809368003A3011F480E408
:1003000005C03C3011F080E004C080EC80936A00AE
:100310008FEFDF91CF91089580E287BB88BB80E0AB
:1003200090E034D38F3F09F081BFBC9A20E083EB8B
:1003300091EF0197F1F72F5F2431C9F7BC982EE0B8
:1003400088E190E00FB6F894A89581BD0FBE21BD5D
:100350004FD07894A89578D0FDCFDF92EF92FF929E
:100360000F931F93CF93DF9300E030E8D32EC0E0CC
:10037000D0E01D2D100F11BF98D17C0184E3E81649
:1003800089E0F8060CF0102FD6942196C830D105DC
:1003900011F0012FEECF012F115011BF1F5F13C0BD
:1003A00084D19C012453394037FF03C030952195F7
:1003B0003F4F2E153F0514F0970101C011B781B7CB
:1003C0008F5F81BF790121B730E0802F90E00196E7
:1003D000821793072CF711BF61B780E090E0DED25F
:1003E000DF91CF911F910F91FF90EF90DF900895D3
:1003F000AB9A8BB780628BBF8BE4809381008AE5D8
:100400008093800008951F93DC01162F8091800057
:1004100084FF07C08091810098E88927809381003C
:1004200003C08AE580938000912FE2E8F0E08D918F
:1004300081939150E1F782E890E0612F32D11C5F07
:10044000109380001F9108951F93CF93DF936091C5
:100450009100635067FDA5C080918E00CCE0D0E094
:10046000C81BD109CB56DF4F80918D008D3209F02A
:1004700086C0683009F093C083EC809375008AE5EC
:1004800080936100109274008881807639F0CE01EB
:10049000C6DE282F8F3F09F461C067C09A81109291
:1004A0007E008981882321F410927F0022E04FC0D2
:1004B000853019F49093920049C0863099F58B816C
:1004C000813041F488E390E09093900080938F0016
:1004D00022E124C0823041F48AE490E090939000BD
:1004E00080938F0029E11AC08330B9F48A81882370
:1004F00041F48EE190E09093900080938F0024E08F
:100500000DC0813051F0823041F482E290E090934E
:10051000900080938F0026E101C020E080E480936A
:10052000740023C0883021F421E084E990E011C0F8
:10053000893019F49093940009C08A3011F421E0B5
:1005400006C08B3019F48BE48093810020E08EE7A5
:1005500090E09093900080938F0007C0888187FD82
:100560002E8180E88093740006C08F81882319F45F
:100570008E81821708F0822F8093620010C08091D4
:10058000740087FF0CC0CE01F4DD8F3F21F48EE1B3
:100590008093610004C0882311F0109262001092D1
:1005A00091008091610084FF4CC0809162008F3F78
:1005B00009F447C0182F893008F018E0811B809398
:1005C00062008091750098E8892780937500112357
:1005D00031F18091740087FF08C086E790E0612FB9
:1005E000B3DD182F893038F51AC0E0918F00F091F3
:1005F000900086FF09C0912FA6E7B0E084918D930B
:1006000031969150D9F707C0912FA6E7B0E08191BC
:100610008D939150E1F7F0939000E0938F0086E77F
:1006200090E0612F3ED0612F6C5F6C3041F08FEF16
:100630008093620004C08FEF809362006EE160934C
:10064000610094E186B3887131F49150D9F710922A
:10065000920010928C0010E0992309F411E080912F
:100660007300811729F0112309F477DE10937300CA
:10067000DF91CF911F910895A82FB92F80E090E0CE
:1006800041E050EA609530E009C02D9182279795AE
:10069000879510F084279527305EC8F36F5FA8F325
:1006A0000895EADF8D939D930895A6E08827992702
:1006B000AA9569F00197E1F3B499FCCFB49BFECF02
:1006C00081E09927A6B3019611F0A871D9F7089592
:1006D000CF93CFB7CF93C395B49BE9F7B49B0BC02F
:1006E000B49B09C0B49B07C0B49B05C0B49B03C0B6
:1006F000B49B01C0D5C00F92DF93C0918E00DD275F
:10070000CB56DF4F012EB49B03C0DF910F90E6CF95
:100710002F930F931F934F932FEF4F6F06B304FB4D
:1007200020F95F933F9350E03BE065C016B301268C
:10073000502954FDC89556B3012704FB25F92F73A2
:1007400006B3B1F05027102714FB26F906B2223069
:10075000F0F000C016B3012704FB27F90126502949
:1007600006B22430E8F54F77206816B30000F6CFC4
:1007700050274F7D206206B2102F000000C006B344
:1007800000265029102714FB26F906B2E2CF4F7B32
:1007900006B3206400C0DACF01265029187106B2D2
:1007A00069F14E7F2160012F16B328C00026502921
:1007B0004D7F06B22260102F29C0012650294B7FA1
:1007C00006B22460012F2DC016B301265029477FA1
:1007D0002860000006B22EC04F7E06B3206130C0F4
:1007E000422706B3499300265029102706B24FEF3F
:1007F00014FB20F9297F16B379F2187159F10126FB
:10080000502906B2012704FB21F9237F06B371F2B8
:10081000002650293150D0F006B2102714FB22F9DF
:10082000277E16B351F201265029012704FB06B298
:1008300023F92F7C49F2000006B3102714FB24F99A
:100840000026502906B22F7939F270CF10E21ABF74
:10085000002719C03B503195C31BD04010E21ABF8E
:100860000881033C09F10B34F9F020918C001981C7
:10087000110F1213EDCF4A81441F093651F10D3289
:1008800011F0013E29F7009393003F915F914F9142
:100890001F910F912F91DF910F90CAB7C5FD1BCF0C
:1008A000CF91CFBFCF91189520919300222369F368
:1008B00010919100112379F534307AF13093910041
:1008C00020938D0010918E003BE0311B30938E0001
:1008D00024C0009191000130F4F40AE54F7049F40E
:1008E0003091610034FD1AC000936100C5E7D0E08B
:1008F00019C03091800034FD11C000938000C1E820
:10090000D0E010C0052710E000C021C0052710E08E
:10091000C89508BB14C03AE501C032ED032EC0E013
:10092000D0E032E017B31861C49A08B317BB58E19E
:1009300020E84FEF20FF052708BB279517951C3FA0
:1009400028F700004552B0F720FF0527279508BB80
:1009500017951C3FB8F629913A9561F7077E1091DB
:100960009200110F08BBC250D04011F010938C00C0
:1009700010E21ABF006117B3177E402F477E54E084
:100980005A95F1F708BB17BB48BB7FCFE199FECF63
:100990001FBA8EBBE09A99278DB30895262FE1994F
:1009A000FECF1CBA1FBA8EBB2DBB0FB6F894E29ACD
:0C09B000E19A0FBE01960895F894FFCF65
:0409BC00325AFF00AC
:00000001FF
